:030000000219FDE5
:03000B000200AA46
:03002B0002015F70
:03005B000202F5A9
:030073000202DBAB
:1000800002030406080C10182030406080040608A3
:100090000C10182030406080A0C000070F1F3F0DDB
:1000A0000D0403060D0502030202C2AFC0D0C0E07A
:1000B000206217E5256002E473E525F4F58A758B67
:1000C00000D262D0E0D0D0D2AF3285268AC262E5BB
:1000D00026F4602F758B00D0E0D0D0D290D291D290
:1000E00092D2AF32D290D291D292206E0C20660979
:1000F000740AD5E0FDE57E4290758B00D0E0D0D04B
:10010000D2AF32758A00C28DD26201F901B930686E
:1001100005206602C29001B9306805206602C291CE
:1001200001B9306805206602C29201B9C2933068F5
:100130000A2066077428D5E0FDC29001B9C2943048
:10014000680A2066077428D5E0FDC29101B9C295FE
:1001500030680A2066077428D5E0FDC29201B9C252
:10016000AFC2AD53E6EFC0D0C0E0D2D3D2AFC2CE63
:10017000E52A6007207449152A21C07800790020FB
:10018000742EE580307E01F430E70278FF53DACF39
:10019000207E0343DA20307E0343DA10C2D8C271D6
:1001A000E580307E01F430E70279FFC3E89970CB37
:1001B000306103752A40207403752A40885FD2702D
:1001C00020740DE52B6004152B21D043DA01C2D831
:1001D00020700221E3A85F206102C2702074022116
:1001E000E188227882B60403852224C3E525944061
:1001F0004002D26420CF0AD0E0D0D043E610D2AD86
:1002000032C2CF053A7802E52A6005307402152A19
:10021000C3E55F94014005756200412D756300756B
:100220006C00E5622401F56250037562FF7982B7C4
:10023000020D306D1DC3E52294324016854D2279A2
:1002400082B7030E306D0BC3E52294324004798EE1
:100250008722C3E5239522600840041523416105E8
:1002600023D8CA056CE56C7002156CD56D63756D8D
:10027000017805C3E56C956E4057C3E56C956F50EA
:10028000087801756D03020295C3E56C9570500501
:100290007801756D01C3E5659524401E7982B70428
:1002A0000241C6206D14852465E56C046003856EEB
:1002B0006C756D0175233C0202D1E565285005750A
:1002C00065FF41C6F565E5650470067563FF756CED
:1002D000FFD0E0D0D043E610D2AD32C2AFC0D05391
:1002E000E67FC26075910085569485579575910497
:1002F000D0D0D2AF32C2AF53E6EFC2ADC0D0C0E073
:10030000C0F0D2D3D2AFA8FBA9FCC2D83071026131
:100310005C53DACF207E0343DA10307E0343DA20C9
:10032000D271E580307E01F420E7026133882789AD
:1003300028A13B53DACF207E0343DA20307E0343EB
:10034000DA10C2D8C271307402A1277800E580307B
:100350007E01F430E702A127885FA10F53DACF2096
:100360007E0343DA20307E0343DA10C2712061023B
:10037000813553DACF207E0343DA10307E0343DA2F
:1003800020C2D8D271885A895BC3E89558F8E9959C
:1003900059F97B007E087A00C3E8948CE9940050F8
:1003A00005755E008127882178A2E6A8216055C3E3
:1003B000E894C8E994005008E4D2E4FB7A0A810288
:1003C000C3E89468E994015008E4D2E3FB7A0F8112
:1003D00002C3E894D0E994025008E4D2E2FB7A1E0A
:1003E0008102C3E894A0E994055008E4D2E1FB7AC5
:1003F0003C8102C3E89498E994085008E4D2E0FBF9
:100400007A787E00C3E8955CFCE9955DFD30E70AEB
:10041000ECF42401FCEDF43400FD755E00C3EC9AAD
:10042000ED9E5003755E01885C895D855A58855B39
:10043000597802A10FC3E89527F8E99528F9307C8F
:100440000281F3307B0281F3307A0281EC20750265
:100450008158E9FDE8FC8177E9C313F9E813F83026
:10046000790281ECE9C313F9E813F830780281ECE2
:0F047000E9C313FDE813FC206126C3EC941CEDD7
:10047F0094024002818EED7018C3EC94C85012059F
:10048F0029C3E529940A5002A127755F00D270A1F4
:10049F0027E529600215297400207F037896E6244A
:1004AF00FAFEE43400FFC3EC9EFCED9FFD5006788E
:1004BF0000790081F3C3EC94FFED9400400678FFC0
:1004CF00790081F3EC8575F0A4C5F0A2F733F879C4
:1004DF0000400302050F78FF790002050FE9C313EF
:1004EF00F9E813F8307C0EE9600278FFC3E813389F
:1004FF00F8E43400F9C3E894FFE99400400278FF70
:10050F00885FD270206102A127741FF4552F4BF51D
:10051F002FC274EB7002D274752A40307403752A9F
:10052F000A306102A13B20740353DAFE2074037575
:10053F002B20D0F0D0E0D0D0D2AD43E610327901ED
:10054F0002056B790302056B790A02056B791E02AE
:10055F00056B796402056B79C802056B7817E4D5D2
:10056F00E0FDD8FAD9F6227A147B780205927A1038
:10057F007B8C0205927A0D7BB40205927A0B7BC8B5
:10058F000205927902B27DE4C294D5E0FDC291D505
:10059F00E0FDD291D5E0FDD294D5E0FDC290E57695
:1005AF00D5E0FDD2907496D5E0FDD9D9EAF8D5E023
:1005BF00FDD8FBDBCEC29422C37C007D0075F0001A
:1005CF0005F0EA33FAEB33FB50F6EB13FBEA13FAC1
:1005DF00C3E9FFE8FEE89AF8E99BF95004EFF9EE5A
:1005EF00F8B3EC33FCED33FDD5F0DFEDF9ECF82289
:1005FF00E889F08A20D2D4F8A9F07B0030F70B7B82
:10060F00FFF42401F8E9F43400F9E88520F0A4ADF3
:10061F00F0F8E98520F0A4AFF0FEED2EF974003F5D
:10062F00FA7C04C3EA13FAE913F9E813F8DCF48B44
:10063F00F030F70AE8F42401F8E9F43400F9E88916
:10064F00F0C2D4F8A9F0227882B604030206F5C3EB
:10065F00E55F9419401EE52D54067018206D36780D
:10066F00057994E7146007780A1460027812C3E5DD
:10067F004198401F306D09856765756CFF756D0179
:10068F00852224E4F545F546F547F548F549C26D51
:10069F000206F5D26D7994E7147013E523F4333322
:1006AF00F913F8E9540104F9E854FE0206E9E714D6
:1006BF00147014E523F4333333F913F8E9540304B6
:1006CF00F9E854FC0206F1E523F433333333F9131D
:1006DF00F8E954070404F9E854F8C39440F8E9948E
:1006EF0000F98845894622C3E54113F9E54013F81F
:1006FF00C3E54598F8E54699F9500CC3E89480E9AD
:10070F0094FF401602072DC3E8947FE9940050032D
:10071F0002072D787F790002072D788079FF884AAC
:10072F00894B22E54A2547F8E54B3548F9854B209B
:10073F00E4300701F43549FA30E709C3EA94F04091
:10074F001502076BC3EA940F500302076B78FF790A
:10075F00FF7A0F02076B780079007AF0C3E52495D2
:10076F0064500AC374019524500B020789E54B208E
:10077F00E70E020789E54B30E706884789488A4923
:10078F002278A4E6FAC3E54A33F8E54B33F9B1FF13
:10079F00E930E70BC3E89480E994FF4013E1C3C34A
:1007AF00E8947FE994005002E1C3787F7900E1C3B8
:1007BF00788079FFE820E715C3E52398F84009C34F
:1007CF00E8940140030207EA78010207EAE8F424FB
:1007DF00012523F840030207EA78FF884C2278A509
:1007EF00E6FAA848A949B1FFE930E70CC3E894013C
:1007FF00E994FF401602081EC3E894FFE9940050E5
:10080F000302081E78FF790002081E780179FFE9BC
:10081F0020E715C3E54C98F84009C3E8940140035D
:10082F000208457801020845E8F42401254CF840F8
:10083F000302084578FF88242278FFC26420693DAF
:10084F00206A12D264C3E541940A4009C3E5259496
:10085F00405002C26479A1E76023E541601F74FF35
:0F086F008541F0848539F0306A0375F005A4F8EF
:10087E00C5F0600278FFC3E895675002A8678866E6
:10088E0022C3E5409440E5419401E566500314010E
:10089E00A0046002F566227883E6F520120F3F75FC
:1008AE00E89012054D75E890E5E820ECFBA8BDA98F
:1008BE00BE120FD9757130757200C3740013FD74BA
:1008CE0030606613FC74302CFC74003DFDECFAEDC8
:1008DE00FBC3E89AE99B4014E5712430F571E5728B
:1008EE003400F572EA2CFAEB3DFB80E5AE71AF7287
:1008FE00C3E57213F9E57113F8C3E913F9E813F8B8
:10090E007A03C3E913F9E813F8DAF7AA201A700983
:10091E007571007572000209371AEA6008EE28FE3A
:10092E00EF39FFDAF88E718F722275E89022788394
:10093E00E6FFE5E820ECF7A8BDA9BE0573C3E57395
:10094E0094084052757300E9FA79A0E76044EA70A2
:10095E0007E574601B020972C3E895746010E574B4
:10096E005006600C1402097E0460F902097EE574DB
:10097E00F574C3946D401B7564C0C3940440137525
:10098E006480C39404400B756440C39404400375A3
:10099E00640075BB0622EFC39401601F7430601BA8
:1009AE00C3E894FFE994035012C3E89571E9957278
:1009BE005009E564600C15640209D0E564F4600228
:1009CE000564A864C3E524985002A824C3E895657D
:1009DE00400AA865E565F460038565648825882668
:1009EE00E573B4070375BB1022743279A687F0A4A1
:1009FE00C5F0A2F733F8C3E895644002A8648822D4
:100A0E008824882588268867227540007541F02243
:100A1E00C2AF75C820A8CCA9CDAA3A30CF010A75AD
:100A2E00C824D2AFAB3BAC3C883B893CC3E89BF8B7
:100A3E00E99C206908F930670261334190AD3D8A27
:100A4E003DF9EA9DFA600478FF79FFAE3EAF3F8B29
:100A5E003E8C3FC3EC9FFCC3E99CF542A83BA93CEE
:100A6E00C3E89EF8E99FF9C3E54113FBE54013FA8D
:100A7E00E82AF540E93BF54150067540FF7541FF08
:100A8E0041DAAA40AB41AC40AD417E047F02C3EBDC
:100A9E00940440021E1FC3EB940840021E1FC3EDB8
:100AAE0013FDEC13FCDEF7C3EA9CFAEB9DFBEF6043
:100ABE0009C3E913F9E813F8DFF7EA28FAEB39FB73
:100ACE008A408B4150067BFF8B408B41C3EB9402D7
:100ADE005002D2673069047F0361057892E6FFC346
:100AEE00E537948240110FC3E53794A040010FC340
:100AFE00EF940640027F057E07E541C4540FF9E5E9
:100B0E0041C454F0F8E540C4540F28F8C3E89EFAE7
:100B1E00E99400FB4009C3EA9402EB940050047A76
:100B2E0002E4FB617FAA40AB41EBC4FEEAC4540F62
:100B3E004EFCC3EA9CFAEB9400FBC3E813C313F814
:100B4E00EA28FAEB3400FB8A408B41C3EB94024057
:100B5E0002C2677807EBC4FE7B00EAC4540F4EFA5C
:100B6E00C3EA98FA4005C3940250027A027892E6DC
:100B7E00FF306002617F855256855357D26043E63F
:100B8E0080C3E49AF8E49BF93067028119E8FAE928
:100B9E00FBD3E913FDE813FC88528953C3EF94038A
:100BAE006038EF20E00DE82CF8E93DF9ECFAEDFBAA
:100BBE00020BD4E828F8E939F9C3E82402F8E9343D
:100BCE0000F97AFE7BFFC3EF9403400E8A548B55D7
:100BDE00884E894F8C508D51814D885489558A4E3F
:100BEE008B4F8C508D51306920C3E53394034019DF
:100BFE00E542A2E713F8E555F4240138400B20E74F
:100C0E00087554FFF42401F555814DE8FAD3E81325
:100C1E00FC8852C3EF94036020EF20E007E82CF825
:100C2E00ECFA8139E8282402F87AFEC3EF940340E7
:100C3E00088A54884E8C50814D88548A4E8C50E5CB
:100C4E006BC3335002646BF56B30600281577534A1
:100C5E0002D26043E680E52D54066026A840A941E5
:0F0C6E00C3E913F9E813F8C2AF53E67F7591009D
:100C7D00C3E498F594E499F595759104D26043E633
:100C8D0080D2AF22D265754400752000306B03759C
:100C9D002040020CB0D265754400752040306B03C6
:100CAD00752000D2AF7801206722E52D5406600231
:100CBD00C265C3E541940540137802940540087858
:100CCD0003940540027806306902780A206019E520
:100CDD0044601530690AC3E53394034003D53406E7
:100CED00D2AFD26CA182915FD2AF0000C2AF2067AC
:100CFD0026E541C3FB940F40027B0FEB24053073B7
:100D0D000123306A02742820620123F930690279C7
:100D1D0082E58BC39940B50544E59BF45440B5205D
:100D2D0002A16C30690A08C3E8940A40010881D910
:100D3D0020650281B0C26553E67F75910030671062
:100D4D007594007595FE759104D26043E68081B06F
:100D5D00AE40AF41C3E49EF594E49FF595A153C316
:100D6D00E5339402500281B030650281B0D802A102
:100D7D008081D9C26C53E67F759100855494855559
:100D8D0095759104854E56854F57D26043E680D2B6
:100D9D00AFE52D54066008206A020533020DBC3004
:100DAD006C0D206B0A2065071581158102160C222A
:100DBD0078003064053065027801E53775F007A4D9
:100DCD00F9E5F028F5F0E9A2F013A2F113A2F21360
:100DDD00F537C394785003753778C3E537953840A8
:100DED0008D266D290D291D292306002A1F685508F
:100DFD0056855157D26043E68022207D11C2AF75D2
:100E0D004302C294D293D2AF759F11020FD6C2AFD7
:100E1D00754302C294D295D2AF759F11020FD63091
:100E2D007243207D20C2AF75430390013D757E1046
:100E3D00D292C295306204C291C14AD294D2AF759A
:100E4D009F21020FD6C2AF75430390013D757E10F1
:100E5D00D290C293306204C291C16AD294D2AF755E
:100E6D009F01020FD6207D17C2AF75430390011865
:100E7D00D292306202C291D2AF759F21020FD6C2BB
:100E8D00AF754303900118D290306202C291D2AF78
:100E9D00759F01020FD6207D11C2AF754304C29319
:100EAD00D295D2AF759F01020FD6C2AF754304C262
:100EBD0095D293D2AF759F21020FD6307243207D0C
:100ECD0020C2AF75430590012C757E08D291C29456
:100EDD00306204C290C1E6D293D2AF759F11020F5A
:100EED00D6C2AF75430590014E757E20D291C29446
:100EFD00306204C292E106D295D2AF759F11020FF6
:100F0D00D6207D17C2AF75430590010ED291306288
:100F1D0002C290D2AF759F11020FD6C2AF754305B5
:100F2D00900122D2913062EBC292D2AF759F110225
:100F3D000FD6207D11C2AF754306C295D294D2AFA4
:100F4D00759F21020FD6C2AF754306C293D294D2BC
:100F5D00AF759F01020FD6307242207D20C2AF7552
:100F6D00430190014E757E20D290C293306204C22F
:100F7D0092E182D295D2AF759F01020FD6C2AF75A5
:100F8D00430190012C757E08D292C295306204C245
:100F9D0090E1A2D293D2AF759F21E1D6207D16C2EA
:100FAD00AF754301900122D290306202C292D2AF4E
:100FBD00759F01E1D6C2AF75430190010ED29230FB
:100FCD006202C290D2AF759F21C2662290010C754C
:100FDD007E00D290D291D292C293C294C295C26237
:100FED002278807607087607087601087604087659
:100FFD00FF0876FF08760A08760208760108760162
:10100D00788C76010876000876B40876FF0876FFAE
:10101D000876FF0876030876FF0876010876FF0844
:10102D0076250876D00876780876C808760408768E
:10103D00FF08760108760008767A08760A087601A8
:10104D000876010876000876FF227887E6FFC272DF
:10105D007888C27DE630E102D27DC27E7889E630A5
:0F106D00E102D27EC3EF94026008758E01D27348
:10107C00021084758E00C273227880E61490008072
:10108C009378A4F67881E6149000809378A5F6788E
:10109C0086E61490008D9378A6F6789FE6F870019A
:1010AC0008C3E8941140027811E82828F56E256EE3
:1010BC00256E28F56F256E2828F570789CE6753816
:1010CC00FF75390CB402067538A075390AB40306DD
:1010DC0075388275390578A3E61490009A93F569F2
:1010EC00120FD922227896E6FA7897E6FB7888E6F2
:1010FC00B40305C3EB940EFB307F047A007BFFC373
:10110C00EB9AFCC3948250027C827575000575ECD9
:10111C008575F0A4C3E5F0947D40F222D27F11F1E5
:10112C0012055C7A007B007C10120552E55F2AFAEE
:10113C0074003BFBDCF37C04C3EB13FBEA13FADC1B
:10114C00F7FEC27F11F122E5EF20E60375200005C2
:10115C0020903FFFE520146006901DFF1460009363
:10116C0004600375EF1253D9BF7581C043FF801221
:10117C00054D75EF0243B203E5B3240420E70DF5EA
:10118C0021E5E320E0068521B343E301120FD97575
:10119C0080FF75A40075F19175D47F75900775A5C6
:1011AC003F75F2FF75D50075A60175E241E4F8F6BE
:1011BC00D8FD756B01120FEE121654789886767561
:1011CC003001C2AF12056612057612055C12057D60
:1011DC0012055C12058412055C1217771205661253
:1011EC000566120561C2AF78FA79FA308707D9FB28
:1011FC00D8F7021C001157118511F011F17898865F
:10120C0076120FD975885075891275C8247591049A
:10121C0075D84075A82275B80275E690759B8075D7
:10122C009D0075D10E75BC5875BB0675BA1175E865
:10123C008012054DD2AF1208A553DACF207E03439E
:10124C00DA20307E0343DA1043DA01C2D8C27112BD
:10125C000566D2617B037A0CE55E70077A0CDB03C2
:10126C000211F112055C2070030211F1C270E55FEE
:10127C00C3940240E1E52F541F856160F561B560B0
:10128C00D5DAD5C26153DACF207E0343DA20307E23
:10129C000343DA10C2D8C27178A2E67008D274E5A2
:1012AC002F54E0F52FC275752900120561307409B1
:1012BC00C3E529940A4002D27512055278023074A3
:1012CC00027800C3E55F9840F0C2AF1205761205B4
:1012DC0076120576D2AF120566754D00120552785E
:1012EC008CE6C3940150030213BEE530C394015045
:1012FC00030213BE207435C3E55F94FF5003021341
:10130C00BEC2AF12058BD2AF120561C3E55F94016B
:10131C0050EFC2AF120576120557120576D2AF12F6
:10132C000561C3E55F94FF40E90217FC7F05D27F9E
:10133C0011F1120561C2AFC27F11F1AE5FC3E55F5F
:10134C00947FD2AF407612054DC2AF12058BD2AF4F
:10135C00DFDC3128C3EE94057897F6120566121679
:10136C009612177F7F0AD27F11F1120561C2AFC2AC
:10137C007F11F1AE5FC3E55F947FD2AF50E61205EB
:10138C004DC2AF120576120557120576D2AFDFD6D5
:10139C003128EE24057896F6120566121696121769
:1013AC00AE12056111F1C3E55F94FF5002610002BA
:1013BC0017FCC3E55F954D4003855F4D12056178C1
:1013CC00017988E7B403027805C3E55F98400241D0
:1013DC00E8C2AF12058B12058B12058BD2AF12052A
:1013EC0066753000E4F531F5320531E531F47039CC
:1013FC000532789AE67819146012783214600D78F8
:10140C007D14600878FA146003753200C3E53298D5
:10141C00401715327531B478998676C2AF12058BA8
:10142C00D2AF78988676120561120557E52A7005B9
:10143C0030740221F178012074027806C3E55F98BC
:10144C0040A7120561E52A70030211F1C2AF120F19
:10145C00D9E4F522F523F524F525F526F56AD2AF66
:0E146C007885E6C333F568E4F545F546F547A7
:10147A00F548F549F573F52CF52DF53775730875AB
:10148A00BB1012054D120938E5E820ECFBA8BDA9EE
:10149A00BEE97001F8887412093C75730875BB10AF
:1014AA007887E6FE760211577887EEF6C2AF756442
:1014BA00FF1209F7852264852265852266D2AF75F7
:1014CA00220175240175250175260185636C756DE8
:1014DA00017888E6B40307C27D307602D27DD268ED
:1014EA00D269753300120F3F120F64120A17120ADB
:1014FA001E120A17120A1E120A17021513C2AF1178
:10150A0057D2AF75730075BB06120CA2120656129B
:10151A000DBD120E07120A1E120C91306D0312062F
:10152A00F620670312084830670312088F120DBDB0
:10153A00120E2C120A1E120CA2306D03120732125E
:10154A000DBD120EA3120A1E120C91306D03120762
:10155A0090120DBD120EC8120A1E120CA2306D0393
:10156A001207ED120DBD120F3F120A1E1209381290
:10157A000C91120DBD120F6412093C120A1E306939
:10158A002F206B2C85676485676585636C756D0193
:10159A0079187A0CC3E533994009C269D26A8A3547
:1015AA000215BAC3E55F940140030215130216142B
:1015BA00306A1B206B18E535147004C26AA107F55E
:1015CA0035C3E55F940140030215130216147536FC
:1015DA0000C3E5629401400985676585636C756D92
:1015EA0001C3E56278FA985021307404E52A601A3A
:1015FA0078F0306B058567647820C3E5419850021E
:10160A00A1130536E55F6002C117753600C2AF1235
:10161A000FD97887E6FE760211577887EEF6E4F559
:10162A0022F523F524F525F526F568C268D2AF120E
:10163A00054D120FD9307406E52A700221F1788D12
:10164A00E6C39401400241C561F0901A0D78201258
:10165A0016D8E520B4A50CA31216D8E520B45A036F
:10166A00021676120FEE121696021695901A037843
:10167A00807B0A1216D8A308DBF9901A0F788C7BA4
:10168A00181216D8A308DBF9901A2722C2AF12172C
:10169A00171216F1901A00740E1216DDA3740412B2
:1016AA0016DDA374141216DD901A0378807B0A12D1
:1016BA0016DCA308DBF9901A0F788C7B181216DC5B
:1016CA00A308DBF912172A121708901A2722E493A3
:1016DA00F622E6438F01538FFD75EF0275B7A575A4
:1016EA00B7F1F0538FFE22438F02438F0175EF0249
:1016FA0075B7A575B7F1901A0DF0538FFC22901AA1
:10170A000D74A5D1DD901A0E745AD1DD227A307982
:10171A00D07820901A40D1D8E520F709A3DAF72229
:10172A007A3079D0901A40E7D1DD09A3DAF922ABF1
:10173A0077A878BB01027980BB02027981BB0302D8
:10174A007982BB04027994BB05027983BB060279CC
:10175A0086BB07027992BB08027987BB0902799C8A
:10176A00BB0A027988BB0B027989E8F7227C051249
:10177A000566DCFB22C2AF12057612057D120584CE
:10178A0012058B12055712057612057D1205841271
:10179A00058B12055712057612057D12058412056E
:1017AA008BD2AF22C2AF12058B12058412057D12AD
:1017BA00057612055712058B12058412057D12054E
:1017CA007612055712058B12058412057D120576CD
:1017DA00D2AF22AE77AF78C2AF1205761205761273
:1017EA000576120557DEF212058B120557DFF8D27D
:1017FA00AF22F17F12177712177775770175780183
:10180A007579001217DD7C05AD5F120566C3ED958B
:10181A005F70F5C3E55F9401400AC3E55F94FF403A
:10182A003702183F12173912169612177FC2AF7570
:10183A00EF12121777DCD10579C3E57994035002C8
:10184A0080C11217770578E5771490009F93F808FE
:10185A00C3E57898500280A8121777121777057790
:0F186A00C3E577940C50028094120FEE1216967D
:08187900C2AF75EF12121777E0
:0319FD0002115381
:101A00000E041407070104FFFF0A020101A55A0191
:101A100000B4FFFFFF03FF01FF25D078C804FF01DA
:081A200000FF0A010100FFFFB5
:101A400023506F6C61726973546472323041232089
:101A500023424C48454C4923463333302320202031
:101A60002020202020202020202020202020202076
:101C0000C2AFC2D353D9BF7581C043B20343FF8073
:101C1000752438752503B1C975EF0275E24043F1AB
:101C20008053A47F75D400D2877DFA780379E67C4F
:101C300010752200752300901DD67B0675249875BB
:101C400025013087028142208708D8FBD9F9DCF7CB
:101C500081B4308708D8FBD9F9DCF781B4B189E4C5
:101C600093A3C39A6004DDC381B4DBDBB17B600264
:101C7000812B7B08E493FAA3B15CDBF87A30B15C8A
:101C8000752200752300B17BEAFCEBFDC3ED94FEE9
:101C9000400EB17B8A278B28ED30E0048A828B834B
:101CA000B17B7AC270D8C3ED94FE601350CEBD00F4
:101CB00025EC60097520007521FF0200008100A855
:101CC00027A9280809D804D90281D3B17FEA89AAB3
:101CD000F281C50D81A0C3ED94035049EDA2E092BD
:101CE000007AC5C3E5829400E583941C50902000DF
:101CF00010438F02438F0175B7A575B7F1F030001F
:101D00001FA827A9280809438F01538FFDD804D99C
:101D100002A12089AAE275B7A575B7F1F0A3A10DBC
:101D2000538FFC817C7AC1BD030CE493A3FAB140CC
:101D3000DCF8B138817C817EAA22AB23B15CEBFA5E
:101D4000EA6222752608C3E52313F523E52213F57D
:101D50002250066323A0632201D526EAB1C9B1C986
:101D600075260AEAF4200102D287300102C287B147
:101D7000C9C3134002C201D526EB22B17FEAFB2082
:101D80008702A17F308702A184752608AE24AF2583
:101D9000C3EF13FFEE13FEB1CDB1C9C3EA13308711
:101DA000024480FA30E703632201C3E52313F523DD
:101DB000E52213F52250066323A0632201D526D91C
:101DC000E52265236523F52222AE24AF250E0FDE22
:101DD000FEDFFCD20122424C48656C693437316326
:041DE000F3300601D5
:00000001FF
